:100000000EC026C025C024C023C0E6C021C020C029
:10001000B2C01EC01DC01CC01BC01AC019C0112414
:100020001FBECFEDCDBF10E0A0E6B0E0EEEEF1E0F8
:1000300003C0C89531960D92A036B107D1F710E0F4
:10004000A0E6B0E001C01D92A53AB107E1F701C0FA
:10005000D7CFCFEDD0E0DEBFCDBF86D0B7D088E11F
:1000600090E02FE00FB6F894A89581BD0FBE21BD9A
:1000700087B3876087BB789420916000909161007E
:10008000309162008091630080FF1EC090E0492F94
:10009000392FE5E6F0E02FE38081843610F49F5F8E
:1000A00009C08081853628F08081883C10F44F5F3C
:1000B00001C03F5F2150319627FFEECF242F809162
:1000C00063008E7F80936300313130F088B318BABB
:1000D00088B3856088BB15C0892F869586952817BB
:1000E00020F488B318BAC09A0CC0822F86958695E2
:1000F000981720F488B318BAC29A03C088B318BA04
:10010000C19AA895BFCFCF93DF93282F392F2150C5
:1001100030408FEF2F3F380771F0A0EDB7E0C0E01F
:10012000D0E08A2F9B2F0197F1F7215030408FEFBD
:100130002F3F3807B1F7DF91CF910895282F392F3E
:10014000215030408FEF2F3F380769F042E050E0F8
:1001500060E070E0842F8A95F1F7215030408FEFF6
:100160002F3F3807B9F7089583E987B988E084BB42
:100170008FE886B908951F920F920FB60F9211243F
:100180008F939F93EF93FF93809164008F5F809391
:100190006400803438F010926400809163008160C4
:1001A0008093630080916400E82FFF27EB59FF4F95
:1001B00084B195B1969587958083FF91EF919F913A
:1001C0008F910F900FBE0F901F9018951ABC85E06D
:1001D00083BF82E089BF08951F920F920FB60F92DE
:0E01E0001124369A0F900FBE0F901F901895A5
:00000001FF
